:100000004928A0001C200A302220200880048413E4
:1000100080068C018D01841720088006640080060C
:100020008413000503191A2810088C0703188D0F74
:100030000B288D030D08442880041E28FF3A8417DE
:10004000800544288F018E00FF308E07031C8F0728
:10005000031C442803308D00DF30302024288D011C
:10006000E83E8C008D09FC30031C39288C070318EE
:1000700036288C0764008D0F36280C183F288C1CFE
:1000800043280000432808008313031383126400ED
:1000900008008316FF3085008312850186018316D0
:1000A00086018312FF30900005308400013001206A
:1000B000A500FF3090000530840002300120A6002A
:1000C000FF3090000530840001300120A50064005D
:1000D0000130250203187928FF3090000530840094
:1000E00002300120A600640001302602031888288F
:1000F0006028061464002508003C031960282508C0
:10010000222064002508003C031960280610792885
:10011000861464002608003C031960282608222063
:0E01200064002608003C031960288610882819
:02400E00FD3F74
:00000001FF
